:0200000057297E
:10000800FF00030E8301B0000A08B1008A017008DE
:10001800A2007108A1007C08A0000408A300063013
:10002800B4000730B5000130B600B70113217008DD
:10003800031932282E14A40A2408183A031D252867
:10004800A4010230FB000430FC00BA30FD00FD0BB7
:100058002B28FC0B2B28FB0B2B2800000730B400A7
:100068000730B5000130B600B70113217008031935
:1000780051282E14A80A28083C3A031D4428A80130
:100088000230FB000430FC00BA30FD00FD0B4A28AA
:10009800FC0B4A28FB0B4A2800000830B400073044
:1000A800B5000130B600B7011321700803195D28A7
:1000B8002E142E1C6628A60A2608143A031D662844
:1000C800A6012E103D308100A50A2508143A031D0B
:1000D8006F28A70AA5010B112208F0002108F100DA
:1000E8002008FC002308840031088A00300E8300B1
:0600F800FF0E7F0E09005F
:1000FE00A53083120313FD00FD0B832800000000C2
:02010E000800E7
:0E011000831203132C088A002B0882000800BB
:10011E0083120313F8010830FC00700DF80D7408FB
:10012E00F80203189C28F8070310F00DFC0B942816
:02013E000800B7
:10014000C1283F3083120313F00008000630F0008E
:1001500008005B30F00008004F30F0000800663007
:10016000F00008006D30F00008007D30F00008005D
:100170000730F00008007F30F00008006730F00022
:100180000800831203133208003A0319A128320829
:10019000013A0319A6283208023A0319A92832089D
:1001A000033A0319AC283208043A0319AF2832087D
:1001B000053A0319B2283208063A0319B52832085D
:1001C000073A0319B8283208083A0319BB2832083D
:0801D000093A0319BE280800DA
:1001D80083120313B3013208093C03180E290A30AD
:1001E800F4003208F0008F207008B3007008B300E4
:1001F800B30D3310B30D3310B30D3310B30D3310EB
:100208000A30F4003208F0008F207808F0007008F7
:0E021800B30410293208B3003308F0000800C8
:1002260083120313B9013508F1000130F00071089B
:1002360003192129F00D7010FF3E1B297008B80024
:10024600340884000008F00570080130031D0030F2
:10025600F0003708F006031948293608003C031851
:1002660038297F207F20B6033029340884003808D7
:100276000005F00070080130031D0030F00037085B
:10028600F00603194829FF30B9003908F0000800C4
:1002960088208A110A128000840AAB0A0319AC0A64
:0802A600F003031D4B290800C1
:1002AE0083120313A401A501A601A701A8018501CC
:1002BE0009108910063083169F008312860187016C
:1002CE00880183168501803086008030870080305B
:1002DE00880009108910573081003D30831281004B
:1002EE008B178B162E1427083C3A031D8029A80A5B
:1002FE00A70128083C3A031D8629A40AA801240850
:10030E00183A031D8B29A4012E1CDC2989142808F8
:10031E00B200EC207008A9000F307005F1007108D2
:10032E00AA00F0307005AD00AD0CAD13AD0CAD13E1
:10033E00AD0CAD13AD0CAD137108B200A02070085A
:10034E0088002D08B200A020700887002408B20093
:10035E00EC207008AF000F307005F1007108AA0094
:10036E00F0307005AD00AD0CAD13AD0CAD13AD0C92
:10037E00AD13AD0CAD137108B200A020700886004D
:10038E002D08013A031DD0292D08B200A0207008B7
:10039E0085002D08023A031DD6293B3085002D0815
:1003AE00003A031DDB298501E129850186018701BC
:1003BE00880189012408023A031DEE292808013A12
:1003CE00031DEE292708003A031DEE2909142408FF
:1003DE00023A031DFB292808013A031DFB292708B1
:1003EE00013A031DFB29091024080F3A031D082AA0
:1003FE002808193A031D082A2708003A031D082A5F
:10040E00091424080F3A031D152A2808193A031D4A
:10041E00152A2708013A031D152A09107A29162ACA
:02400E00422F3F
:00000001FF
